:0200000480007A
:100000006F008004732F2034930F80006308FF0378
:10001000930F90006304FF03930FB0006300FF038E
:10002000130F000063040F0067000F00732F2034CC
:1000300063540F006F00400093E19153171F0000BD
:1000400023223FFC6FF09FFF93000000130100008C
:10005000930100001302000093020000130300004C
:100060009303000013040000930400001305000034
:10007000930500001306000093060000130700001C
:100080009307000013080000930800001309000004
:1000900093090000130A0000930A0000130B0000EC
:1000A000930B0000130C0000930C0000130D0000D4
:1000B000930D0000130E0000930E0000130F0000BC
:1000C000930F0000732540F16310050097020000B4
:1000D000938202017390523073500018970200000F
:1000E00093824202739052309B021000939252030B
:1000F0009382F2FF7390023B9302F0017390023AF5
:100100007350403097020000938242017390523046
:10011000735020307350303093010000970200007C
:10012000938282EE73905230130510001315F5017F
:10013000635C05000F00F00F930110009308D005D9
:10014000130500007300000093020000638A0200A0
:1001500073905210B7B200009B82921073902230BD
:100160007350003097020000938242017390123462
:10017000732540F173002030B70001009B8010F020
:1001800093900001938000F013F7F0F0B7030100A3
:100190009B8313F093930301938303F09301200057
:1001A0006318771CB710F00F9B8000FF13F7000F48
:1001B0009303000F93013000631C771AB700FF0010
:1001C0009B80F00F13F7F0709303F0009301400051
:1001D0006310771AB7000F009B80F00F9390C00058
:1001E0009380F00013F7000F930300009301500079
:1001F00063107718B70001009B8010F09390000106
:10020000938000F093F0000F9303000093016000CF
:100210006390701613020000B710F00F9B8000FF70
:1002200013F7F0701303070013021200930220006B
:10023000E31452FE9303007093017000631A73126B
:1002400013020000B700FF009B80F00F13F7000FB0
:100250001300000013030700130212009302200092
:10026000E31252FE9303000F930180006312731098
:1002700013020000B7000F009B80F00F9390C000A6
:100280009380F00013F7F0F013000000130000005B
:10029000130307001302120093022000E31C52FC18
:1002A000B7030F009B83F30F9393C3009383F30073
:1002B00093019000631E730A13020000B710F00F41
:1002C0009B8000FF13F7F0701302120093022000CE
:1002D000E31652FE930300709301A000631A77089F
:1002E00013020000B700FF009B80F00F1300000016
:1002F00013F7000F1302120093022000E31452FEC2
:100300009303000F9301B0006314770613020000FB
:10031000B7000F009B80F00F9390C0009380F00017
:10032000130000001300000013F7F0701302120016
:1003300093022000E31E52FC9303F0009301C000DF
:10034000631877029370000F930300009301D000AD
:1003500063907002B700FF009B80F00F13F0F07005
:10036000930300009301E0006314700063103002F7
:100370000F00F00F638001009391110093E11100D1
:100380009308D00513850100730000000F00F00FE3
:10039000930110009308D0051305000073000000BE
:1003A000731000C00000000000000000000000000A
:0C03B00000000000000000000000000041
:1010000000000000000000000000000000000000E0
:1010100000000000000000000000000000000000D0
:1010200000000000000000000000000000000000C0
:1010300000000000000000000000000000000000B0
:081040000000000000000000A8
:040000058000000077
:00000001FF
